:1000000009298030A100FE30A7200130A7207530DB
:10001000A7003030BF28A101A117AF00AF08031D12
:100020001328030114280130AF020310A20CA20C04
:10003000A20CC0302205403EAF07FE30A7202F089B
:10004000A728A101A117AF00FE30A7202F08A728DD
:10005000A401AA00AB01A01124080319A0150530C2
:10006000A3002730A900103041200330A900E83058
:100070004120A90164304120A9010A3041202A0809
:100080004828A8002B08A7002A08A600D320260885
:10009000A600A3030319A011240803195228230260
:1000A000031859282608031DA011A0195928303E0D
:1000B000A7280800AD0006118611831606118611C7
:1000C0000F30860583122D08A01884283E30A70023
:1000D0008030BF203330AC0098201330A700883028
:1000E000BF2098206430BE2098206430BE2022308B
:1000F000AC009820283083200C30832006308320E9
:10010000A0142D0884282014AC00201C92288611ED
:10011000033C031C972897200730A700D030BF204E
:10012000031408002014FE3C0319A5288615201C82
:10013000201006150F3086052C08F03986040611AC
:10014000AC0E201898283230BE202D080529A11B9E
:100150005A28080083178001840AFF3E031DAB283C
:100160000529A901A800FF30A807031CA907031C43
:1001700005290330A700DF30BF20B328A701E83EE0
:10018000A600A709FC30031CC828A6070318C52829
:10019000A6070000A70FC5282618CE28A61CD2281F
:1001A0000000D2280800AB01AA011030AC00270DD6
:1001B000AA0DAB0D2808AA022908031C290FAB02BF
:1001C0000318E9282808AA0729080318290FAB07EC
:1001D0000310A60DA70DAC0BD72826080529103053
:1001E000B000A701A601AD0CAC0C031CFD2828082B
:1001F000A60729080318290FA707A70CA60CAB0C04
:10020000AA0CB00BF3282A080529831383120313C1
:100210000800A00107309F00E03083168500FF3002
:1002200086008113831285018601203084006030AE
:10023000AB20A03084005030AB2020308400303020
:10024000AA20C830B120012077305A205A205A20E5
:100250002E305A2070305A2069305A2063305A208C
:1002600062305A208030A100C030212061305A20F5
:1002700073305A2069305A2063305A202E305A2069
:100280006E305A206C305A200B30A900B830B220A2
:10029000012044305A2043305A2046305A20313011
:1002A0005A2036305A204E305A204C305A20463090
:1002B0005A208030A100C230212056305A202D30E3
:1002C0005A2032305A200730A900D030B220012005
:1002D0004C305A2044305A2052305A2020305A2074
:1002E00061305A2066305A2072305A2065305A20C8
:1002F0008030A100C030212067305A2065305A205C
:100300006C305A2065305A206E305A2086188E295B
:10031000851F8C2905148D2905108629012053304D
:100320005A2069305A2067305A206E305A20613086
:100330005A205A206C305A208030A100C030212031
:100340007A305A206F305A2065305A206B305A204C
:1003500065305A206E305A204914831605128312D4
:1003600005123E2AC2013B03A500C8014808250228
:10037000031CCA29ED21C91CC7294808A200A601EF
:10038000A20A0314A60DA20BC2292608C204C80A99
:10039000031DB6294208B100B201B20CB10CB20C77
:1003A000B10CB20CB10CB20CB10C0F30B20531086B
:1003B000AC003208AD000A30A800A901EF20B1005E
:1003C0002B08B2004208B300B4010F30B30500306F
:1003D000B40531083307C2000800B801B901061896
:1003E000022A0130B120B80A0319B90A0B303902C8
:1003F000031C012A031D002AB9303802031C012AFC
:100400006F2CEF299B30B1208310061883148318BA
:10041000C914831CC910491C212A4308B100B20128
:100420000310B10DB20DB10DB20DB10DB20D310809
:10043000A6003208A7003A30A800A901D320BC00CA
:10044000342A8030A1000230A2003C080D20023086
:10045000A4004308292003014919013EC918013AA3
:1004600003194911031D4915C30A85140130A90058
:10047000F430B2208510F030B1200800BA01C30179
:100480004912491ADC2AB801B901061C582AB80ACF
:100490000319B90A0130B120AF303902031C572AC1
:1004A000031D562AC9303802031C572A6F2C452ACF
:1004B000B801B9010618942AB80A0319B90A0A3012
:1004C000B1204918882A38080B3A3904031D732AC9
:1004D0008030A1000230A2003C080D2035305A20A7
:1004E00039305A20872A3808193A3904031D7A2AE4
:1004F0008514872A38084B3A3904031D812A851050
:10050000872A3808FA3A3904031D872A6F2C932A60
:1005100011303902031C932A031D922A95303802A8
:10052000031C932A6F2C5A2A41303A02031C992A41
:100530006F2CBA0AB908031DA12A65303802031CC2
:10054000A22A4916491CDB2A3A08B100B20103105D
:10055000B10DB20DB10DB20DB10DB20D3108A60045
:100560003208A7004130A800A901D320BC00803088
:10057000A100212053305A2069305A2067305A2078
:100580006E305A2061305A205A206C305A20203068
:100590005A20C030212067305A2065305A207630EA
:1005A0005A206F305A206E305A2064305A206530FD
:1005B0005A206E305A20412A491C022B0120493012
:1005C0005A206E305A2069305A2074305A206930CF
:1005D0005A2061305A206C305A2069305A208030BD
:1005E000A100C030212073305A2065305A2072306B
:1005F0005A2065305A206E305A202E305A205A2008
:100600005A20652B0130BC000230A2003C080B20B0
:10061000A101C91D1A2B3B3040020318112BC00A3F
:10062000192BC001173044020318182BC40A192BC8
:10063000C4011E2B4108C0004508C4002D2BC4086E
:10064000031D252B0C30C6002C2B0D304402031C3F
:100650002C2B0C304402C6002F2B4408C6000A3055
:1006600046020318352B20305A208030A10046085E
:1006700028203A305A200230A400400829203A307D
:100680005A2030305A205A20512B0C304402031883
:100690004C2B61305A204E2B70305A200630BC0053
:1006A000532B0730BC000130C008031D0030B500DB
:1006B0001E3040020130031D0030B50401308618A1
:1006C0000301B5040319652B482C491E462CED2166
:1006D0000130C8000F3048020318722BED21C80A00
:1006E000031D6A2B4911C911ED21ED21ED21C91C12
:1006F0007B2B05147C2B05101230C80014304802E7
:100700000318862BED21C80A031D7E2BED2107302F
:10071000BB00B2214208C100ED21491D902BC91533
:100720000630BB00B2214208C500ED21491D992BBE
:10073000C9150630BB00B2214208BD000330BB0022
:10074000B2214208C7000530BB00B2214208BF00F9
:100750000830BB00B2214208BE00ED21491DB12B7B
:10076000C915491CB72BC919B62B49100120C91945
:10077000452C8030A10021203D08282020305A201F
:1007800001303F02031DCB2B6A305A2061305A20C2
:100790006E305A20432C02303F02031DD62B6630A8
:1007A0005A2065305A2062305A20432C03303F02D1
:1007B000031DE12B6D305A2072305A2074305A20BC
:1007C000432C04303F02031DEC2B61305A20703063
:1007D0005A2072305A20432C05303F02031DF72B5C
:1007E0006D305A2065305A2069305A20432C06302B
:1007F0003F02031D022C6A305A2075305A206E3099
:100800005A20432C07303F02031D0D2C6A305A201A
:1008100075305A206C305A20432C08303F02031D9B
:10082000182C61305A2075305A2067305A20432CDA
:1008300009303F02031D232C73305A2065305A20A3
:1008400070305A20432C0A303F02031D2E2C6F308B
:100850005A206B305A2074305A20432C0B303F0200
:10086000031D392C6E305A206F305A2076305A20B2
:10087000432C0C303F02031D432C64305A2065305A
:100880005A2063305A2020305A20472C6F2C3E2AA1
:10089000851F4F2C8316051283120512512C8316C7
:1008A000051683129B30B1200130C008031D0030B3
:1008B000B500013086180301B5040319602C051535
:1008C000851585140130A900F430B2200511851179
:1008D00085100130A9004A30B220C30A682B0120DC
:1008E00047305A2065305A205A206E305A20203026
:1008F0005A2073305A2069305A2067305A2080308D
:10090000A100C03021206E305A2061305A205A2078
:100910006C305A20203084006030AB20A03084003E
:100920005030AB20203084003030AA2083100618CD
:1009300083148318C916831CC91203010618013ECB
:10094000C91A013C031DAA2CB60A0319B70A0130C3
:10095000B1209D2C0301C91A0130013A0319C912B3
:10096000031DC91603010618013EC91A013C031DE7
:10097000BF2CB60A0319B70A0130B120B22C0330DC
:100980003702DE300319360203188A2C49143E2A36
:02099000C82C71
:02400E00503F21
:00000001FF
